:020000040000FA
:040000008FEF00F08E
:020008009ED088
:08001800ECD00C6E960E046E94
:10002000980E056E55D8D8B4CA90D8A4CA80FC0FD3
:10003000D8A0CA92D8B0CA82800E046E960E056E01
:10004000980E086E096ACAB025D8CAB223D842D819
:100050000404CB6E04C006F005C007F000500A6E21
:100060000B6E003C0B6A4BD809500C2E0AD0BE6EAA
:100070000C0EBD6E08BEBD8A08BCBD889394CA84B0
:100080001200BB6E0C0EBA6E08BEBA8A08BCBA88E3
:100090009492F5D700D8D890083205320432120075
:1000A000076A066EFF0E0626072200D0D8A01200AF
:1000B000030E056EE70E02D8F5D7056AFE0F046E33
:1000C000E86A055AD8A012000000040600D0F8D74C
:1000D000096A086A100EF36E0534083609360650B0
:1000E000085C0750095805E30650085E0750095A96
:1000F000D88004360536F32EEFD704501200065090
:100100000A02F3CF08F0F4CF09F007500A02F350C7
:10011000092606500B02F350092608501200F86A0F
:100120004F0EAF6E240EAC6E900EAB6E0001C69AF1
:10013000470E926EE00E936EC00E946E070EB46E74
:100140000F0EC16EA1D09EAA1BD0060EAB1412E1F9
:10015000E1CF44F0E2CF45F0462A1EEE80F0465053
:10016000E126000EE222AECFE7FF44C0E1FF45C02A
:10017000E2FF1100AE50AE50AB98AB8811000AD030
:10018000F2A408D0F294114A122A817A106AD6CFCA
:100190000FF0110011004650475C14E0472AE9CFE8
:1001A00004F0EACF05F00EEE80F04750E926000E8D
:1001B000EA22EF50046E04C0E9FF05C0EAFFD880D0
:1001C000120004D0E868046ED8A012001200466A3B
:1001D000476A9D8A9F8AF28EF28C12009D9A0EEEDB
:1001E00080F0000EEE6AE82EFDD7466A476A9D8AC7
:1001F0001200F29ED8CF5AFEE8CF5BFEE0CF5CFE45
:10020000E9CF5DFEEACF5EFEE1CF5FFEE2CF60FEAA
:10021000D9CF61FEDACF62FEF6CF63FEF7CF64FE80
:10022000F5CF65FEF3CF66FEF4CF67FEA6CF68FE7E
:10023000F28E0001A192D40EB26EB30EB36EF29E96
:100240005ACED8FF5BCEE8FF5CCEE0FF5DCEE9FF83
:100250005ECEEAFF5FCEE1FF60CEE2FF61CED9FF66
:1002600062CEDAFF63CEF6FF64CEF7FF65CEF5FF10
:1002700066CEF3FF67CEF4FF68CEA6FFF28E1000C5
:100280009EA8FED7AD6E1200949A8B9A94988B9884
:1002900094968B9693908A9093928A9294908B9056
:1002A000939A8A9A006A280E066E260E076E020E30
:1002B000B4DE006A280E066E260E076E010EADDE55
:1002C00092988998929A899A92968996336A400E62
:1002D000306E326A230E406E170E436E1D0E426E54
:1002E000620E3F6E060E416E1E0E316E31C03EF044
:1002F0003D6AD8903E363B6AB9EC05F0939A8A8AFB
:10030000320ECEDE939A8A9A2E6A376A60DF66DFF3
:10031000CD6AF294F28A870ED56E820EC06E0E0EF2
:10032000C16E010EC26EB16AA192A082B26AB36AB6
:10033000D08EA292B10EB16E2EDF136EBF0E135C83
:1003400007E3FE0E135C02E370D102D0156A6DD193
:1003500013AE21D0156A8E0E135C05E113C015F0A3
:100360001668176817D09E0E135C05E113C015F0D0
:10037000186819680FD0AE0E135C05E113C015F0B4
:100380001A681B6807D0BE0E135C04E113C015F099
:100390001C681D684AD1155202E147D146D18E0E24
:1003A000155CD8A454D0162803E113C016F04DD024
:1003B00013C017F04050165C18E316503F5C15E36D
:1003C0003B5211E02E86D6CF0FF0D7CF10F03D5024
:1003D0000F24266E3E501020276E000E1120286E2E
:1003E000000E1220296E3C6A2FD04350165C18E391
:1003F0001650425C15E33B5211E02E86D6CF0FF02B
:10040000D7CF10F03D500F24266E3E501020276E9F
:10041000000E1120286E000E1220296E3C6A14D0A6
:10042000780E165C04E137902E908A900DD0790EEC
:10043000165C04E137922E928A9206D07A0E165CF0
:1004400003E137942E948B901668EFD0EED09E0E79
:10045000155CD8A4D1D0182803E113C018F0CAD075
:1004600013C019F01952D8A44CD04050185C18E3AE
:1004700018503F5C15E33B5211E02E86D6CF0FF0AB
:10048000D7CF10F03D500F24266E3E501020276E1F
:10049000000E1120286E000E1220296E3C6A2FD00B
:1004A0004350185C18E31850425C15E33B5211E0CE
:1004B0002E86D6CF0FF0D7CF10F03D500F24266EEA
:1004C0003E501020276E000E1120286E000E1220C4
:1004D000296E3C6A14D0780E185C04E137902E9097
:1004E0008A900DD0790E185C04E137922E928A9290
:1004F00006D07A0E185C03E137942E948B9018681E
:1005000094D04350185C24E31850425C21E30C0E55
:1005100018240D6E0E6A0E3640500D5C416E00EED2
:1005200048F04150EB503B6E3B508218080BD8A46A
:1005300082763B508218100BD8A482783B508218E8
:10054000200BD8A4827A18C03CF02E966ED051D0E1
:100550004050185C1FE318503F5C1CE34050185C8F
:10056000416E00EE48F04150EB503B6E3B5082181C
:10057000080BD8A482763B508218100BD8A482783E
:100580003B508218200BD8A4827A18C03CF02E96DB
:100590004CD02FD0780E185C0DE17F0E195C06E26E
:1005A000780E1A6E19C01BF0E9D803D037802E9050
:1005B0008A801FD0790E185C0DE17F0E195C06E26F
:1005C000790E1A6E19C01BF0D9D803D037822E923B
:1005D0008A820FD07A0E185C0CE17F0E195C06E25D
:1005E0007A0E1A6E19C01BF0C9D803D037842E9426
:1005F0008B8018681AD019D0AE0E155C0AE11A2843
:1006000003E113C01AF003D013C01BF0B7D80DD00C
:100610000CD0BE0E155C09E11C2803E113C01CF0D0
:1006200003D013C01DF050D900D02E52D8B46FD0D3
:100630002EA01BD094C024F095C025F0A0C022F0BD
:10064000A1C023F0D6CF0FF0D7CF10F022500F5C0F
:100650002350105824501158255012581250251864
:10066000D8B0800AD8B850EC05F02EA21BD096C0A6
:1006700024F097C025F0A2C022F0A3C023F0D6CF6B
:100680000FF0D7CF10F022500F5C23501058245099
:1006900011582550125812502518D8B0800AD8B8D1
:1006A00073EC05F02EA41BD098C024F099C025F05F
:1006B000A4C022F0A5C023F0D6CF0FF0D7CF10F002
:1006C00022500F5C235010582450115825501258B6
:1006D00012502518D8B0800AD8B896EC05F02EA68E
:1006E00016D0D6CF0FF0D7CF10F026500F5C275082
:1006F0001058285011582950125812502918D8B0A3
:10070000800A05E78B968B988B9A3B6A2E96D6CFFC
:100710000FF0D7CF10F0385010B601082DE0386A2E
:1007200010B6382A39520CE0898A390639C000F0EF
:10073000280E066E260E076E010E0DEC00F001D09D
:10074000899A3A520CE089863A063AC000F0280E9F
:10075000066E260E076E020E0DEC00F001D0899693
:1007600039503A24016E026A0236015202E1025205
:1007700002E0899801D089889CEF01F0780E1A5C1C
:1007800032E137A02DD02E80D6CF0FF0D7CF10F08A
:100790001B1C036E7F0E03140D6E0E6A0DC002F05B
:1007A000016AD890023601C088F002C089F088C082
:1007B00001F089C002F001500F24226E0250102077
:1007C000236E000E1120246E000E1220256E24C010
:1007D00094F025C095F022C0A0F023C0A1F002D073
:1007E0002E908A9069D0790E1A5C32E137A22DD012
:1007F0002E82D6CF0FF0D7CF10F01B1C036E7F0ECA
:1008000003140D6E0E6A0DC002F0016AD890023614
:1008100001C08AF002C08BF08AC001F08BC002F0E8
:1008200001500F24226E02501020236E000E112062
:10083000246E000E1220256E24C096F025C097F07D
:1008400022C0A2F023C0A3F002D02E928A9234D00C
:100850007A0E1A5C31E137A42DD02E84D6CF0FF05A
:10086000D7CF10F01B1C036E7F0E03140D6E0E6AA3
:100870000DC002F0016AD890023601C08CF002C0AF
:100880008DF08CC001F08DC002F001500F24226E5B
:1008900002501020236E000E1120246E000E122034
:1008A000256E24C098F025C099F022C0A4F023C082
:1008B000A5F002D02E948B901A6812001E681200C8
:1008C000206812001F681200160E1C5CD8A448D0C5
:1008D000400E1D5C06E1396A3A6A8988899A8996D0
:1008E0002AD0400E1D5C15E21D5202E1010E1D6E64
:1008F0001D5040080D6E000ED8A0FF0F0E6ED89050
:100900000D343A6ED8903A36396A898A8996899830
:1009100012D0410E1D5C0FE3C00E1D240D6E0E6A39
:10092000FF0E0E22D8900D34396ED89039363A6ABF
:1009300089868998899A1DC030F039C000F0280E48
:10094000066E260E076E010E0DEC00F03AC000F0A8
:10095000280E066E260E076E020E0DEC00F067D014
:100960001E0E1C5C0FE11DC031F0315205E12E96C8
:10097000640E3D6E3E6A05D031C03EF03D6AD890AF
:100980003E3655D0210E1C5C23E1146A1DBC142A8E
:100990001450325C1CE08B968B988B9A2E96416A91
:1009A00014520AE1E6D8230E406E620E3F6E170E17
:1009B000436E1D0E426E09D04BD9280E406E670E55
:1009C0003F6E1C0E436E220E426E14C032F02FD0CA
:1009D000420E1C5C07E11D5203E1339046D801D062
:1009E000338025D0640E1C5C1EE12E96E86A1DB093
:1009F000010F3BB60108D8A48276E86A1DB2010F48
:100A00003BB80108D8A48278E86A1DB4010F3BBA4C
:100A10000108D8A4827AD8901D343B6ED8903B361A
:100A2000D8903B3604D07B0E1C5CD8B402D81C682E
:100A300012002E902E922E942E968B9A8B988B9637
:100A40003B6A006A280E066E260E076E010E0DEC3C
:100A500000F0006A280E066E260E076E020E0DECE0
:100A600000F0396A3A6A376A12002E6A8B9A8B98BC
:100A70008B968A908A928B90376A396A3A6A3B6A77
:100A8000006A280E066E260E076E010E0DEC00F0B1
:100A9000006A280E066E260E076E020E0DEF00F09D
:100AA00037B003D02E908A901DD0D6CF0FF0D7CF7D
:100AB00010F088C001F089C002F001500F24226EAE
:100AC00002501020236E000E1120246E000E122002
:100AD000256E24C094F025C095F022C0A0F023C05C
:100AE000A1F08170120037B203D02E928A921DD0ED
:100AF000D6CF0FF0D7CF10F08AC001F08BC002F034
:100B000001500F24226E02501020236E000E11207F
:100B1000246E000E1220256E24C096F025C097F09A
:100B200022C0A2F023C0A3F08172120037B403D018
:100B30002E948B901DD0D6CF0FF0D7CF10F08CC055
:100B400001F08DC002F001500F24226E02501020DF
:100B5000236E000E1120246E000E1220256E24C07C
:100B600098F025C099F022C0A4F023C0A5F08270AF
:100B70001200380E486E300E496E280E4A6E200E56
:100B80004B6E100E4C6E080E4D6E4E6A380E4F6E48
:100B9000300E506E280E516E200E526E100E536E97
:100BA000080E546E556A280E566E200E576E100EA3
:100BB000586E080E596E5A6A180E5B6E200E5C6EE7
:100BC000080E5D6E5E6A100E5F6E080E606E616AE2
:100BD000100E626E200E636E646A080E656E666AA1
:100BE000180E676E100E686E080E696E6A6A100E37
:100BF0006B6E080E6C6E6D6A300E6E6E200E6F6E30
:100C0000180E706E080E716E726A180E736E200EDA
:100C1000746E080E756E766A100E776E080E786E1A
:100C2000796A300E7A6E200E7B6E100E7C6E080E86
:100C30007D6E7E6A180E7F6E100E806F080E816FBB
:100C4000826B100E836F846B856B866B876B1200D3
:100C5000380E486E300E496E280E4A6E180E4B6ED6
:100C6000100E4C6E080E4D6E4E6A380E4F6E300EE2
:100C7000506E280E516E200E526E100E536E080EDE
:100C8000546E556A280E566E200E576E100E586E12
:100C9000080E596E5A6A200E5B6E100E5C6E080EBE
:100CA0005D6E200E5E6E100E5F6E080E606E616AE5
:100CB000280E626E200E636E100E646E080E656E56
:100CC000666A676E686A696E6A6A100E6B6E080EF5
:100CD0006C6E6D6A6E6A6F6A706E716E726A736E38
:100CE000746A756E766A100E776E080E786E796A81
:100CF0007A6A7B6A7C6E7D6E7E6A7F6A806B816BAE
:100D0000826B836B846B856B866B876B1200FFD75E
:020000040030CA
:0300010006170ED1
:020005008580F4
:060008000FC00FE00F40E5
:00000001FF
